:10000000301D0020B9160000BF340000951000001C
:10001000951000009510000095100000951000004C
:100020009510000095100000951000005910000078
:10003000951000009510000001100000E73300004B
:10004000B9100000B9100000B9100000B91000008C
:10005000B9100000B9100000B9100000B91000007C
:10006000B9100000B9100000B9100000B91000006C
:10007000B9100000B9100000B9100000B91000005C
:10008000B9100000B9100000B9100000B91000004C
:10009000B9100000B9100000B9100000B91000003C
:1000A000B9100000B9100000B9100000B91000002C
:1000B000B9100000B9100000B9100000B91000001C
:1000C000B9100000B9100000B9100000B91000000C
:1000D000B9100000B9100000B9100000B9100000FC
:1000E000B9100000B9100000B9100000B9100000EC
:1000F000B9100000B9100000B9100000B9100000DC
:10010000B9100000B9100000B9100000B9100000CB
:10011000B9100000B9100000B9100000B9100000BB
:10012000B9100000B9100000B9100000B9100000AB
:10013000B9100000B9100000B9100000B91000009B
:04014000B9100000F2
:100144007BB972B90029BEBF00204FF0004106E020
:1001540008BF00281CBF6FF000414FF0FF3000F0D3
:10016400AFB9ADF1080C6DE904CE002909DB002B11
:100174001ADB00F035F8DDF804E0DDE9022304B011
:100184007047404261EB4101002B1BDB00F028F873
:10019400DDF804E0DDE9022304B0404261EB4101F3
:1001A400524263EB43037047524263EB430300F054
:1001B40017F8DDF804E0DDE9022304B0404261EB06
:1001C40041017047524263EB430300F009F8DDF844
:1001D40004E0DDE9022304B0524263EB43037047B9
:1001E4002DE9F0478C46089D04468A46002B4AD1E7
:1001F4008A42174662D9B2FA82F64EB1C6F1200E8F
:1002040001FA06F3B740B44020FA0EFE4EEA030AA0
:100214004FEA1748230C1FFA87F9BAFBF8FE08FBCC
:100224001EAA0EFB09F243EA0A439A420BD9FB18B1
:100234000EF1FF312CBF012000209A4202D9002880
:1002440000F02A818E469A1AA3B2B2FBF8F008FB9A
:10025400102200FB09F943EA0244A14507D93C19DD
:1002640000F1FF3302D2A14500F210811846A4EB3D
:10027400090440EA0E4000211DB1F4400023C5E901
:100284000043BDE8F0878B4208D9002D00F0F280CE
:100294000021C5E9000C0846BDE8F087B3FA83F1F4
:1002A40000294ED16345C0F0E880824240F2E580E7
:1002B4000846002DE5D0C5E9004AE2E702B9FFDEB1
:1002C400B2FA82F6002E40F099808B1A4FEA124E51
:1002D4001FFA82F801214FEA144CB3FBFEF20EFB25
:1002E400123008FB02F94CEA004CE14508D917EB3F
:1002F4000C0C02F1FF3302D2E14500F2CA801A4627
:10030400ACEB090CA3B2BCFBFEF00EFB10CC08FB5B
:1003140000F843EA0C44A0450ED93C1900F1FF3320
:100324002CBF4FF0010C4FF0000CA04503D9BCF1D9
:10033400000F00F0A8801846A4EB080440EA02402D
:100344009AE7C1F120048B4002FA01FE0CFA01F68F
:10035400E24020FA04F72CFA04FC00FA01F81343F3
:100364003E431F0C320C1FFA83F9BCFBF7F007FB6A
:1003740010CC00FB09FA42EA0C4CE24508D913EB15
:100384000C0C00F1FF3202D2E24500F289801046E3
:10039400ACEB0A0CB6B2BCFBF7FA07FB1ACC0AFBAF
:1003A40009F946EA0C42914506D99A180AF1FF3632
:1003B40001D291457AD8B2464AEA0040A2EB09023A
:1003C400A0FB0E67BA42B446B94602D307D1B04582
:1003D40005D2B6EB0E0C67EB030301389946002DEA
:1003E4006BD0B8EB0C0362EB090202FA04F4CB40C5
:1003F400CA4000211C43C5E9004242E7B740C6F1A8
:10040400200201FA06F3B44021FA02FC4FEA174E27
:1004140020FA02F21FFA87F8BCFBFEF11A430EFB26
:1004240011CC01FB08F0130C43EA0C4C604507D9CE
:1004340017EB0C0C01F1FF3301D2604533D8194698
:10044400ACEB000C92B2BCFBFEF00EFB10CC00FB3C
:1004540008F342EA0C4C634507D917EB0C0C00F186
:10046400FF3201D2634525D81046ACEB030340EAC2
:10047400014130E72946284603E7841A6CEB03035D
:1004840001209A4615E702383C4455E702383C44BB
:10049400EDE6023ABC4433E7AEF1020E3B44D2E649
:1004A40002389C4474E70239BC44C9E7AAF1020A41
:1004B4001A4481E70238BC44D7E72946E1E600BF85
:1004C400704700BF2DE9E04F2746A046A146A2464B
:1004D400A346A4462DED108B4FF0000545EC185BA8
:1004E40045EC195A45EC1A5A45EC1B5A45EC1C5A72
:1004F40045EC1D5A45EC1E5A45EC1F5AF1EE105AB4
:100504004FF66076C0F6FF763540E1EE105A84F37C
:10051400008825462646A447BDEC108BBDE8E08F35
:1005240082680C4B9A60036883F38888436883F37A
:100534008988027B02F00101EFF3948323F0030323
:10054400920748BF43F0020309B143F0010383F368
:100554009488704700ED02E0084AD36848B123F458
:1005640000531B041B0C43F0BF6343F40033D360FC
:1005740070479BB243F40053F5E700BF00ED00E081
:10058400084AD36840B19BB243F4804343F0BF634D
:1005940043F40033D360704723F480431B041B0CE3
:1005A400F4E700BF00ED00E0084AD36840B19BB215
:1005B40043F0080343F0BF6343F40033D360704750
:1005C40023F008031B041B0CF4E700BF00ED00E05C
:1005D400034AD2F88C3043F44063C2F88C3070473D
:1005E40000ED00E0084B1A6818B142F001021A60ED
:1005F400704722F001021A601A6811B142F0020237
:10060400F5E722F00202F2E7D0ED00E00B680133D7
:100614000B60014B1B681847702600202DE9F04F32
:1006240085B00E9C9B46012CB8BF0124012B0CBF46
:100634003023202315468046894601260A270022B6
:10064400DFF870A0019402930AF101040AB9AA45E3
:100654001ED2B5FBF4F049463030C04701220136C2
:10066400B5FBF4F10A23013F012F04FB1155BAFB3A
:10067400F3FAE9D1494605F13000C047BBF1030F55
:1006840003D1019B9C1B002C0FDC05B0BDE8F08F4F
:10069400019BBB42E4DBBBF1020FE1D8494602985F
:1006A40003920136C047039ADAE749462020C0473F
:1006B400013CE8E7FFC99A3B014B1860704700BF53
:1006C40070260020002313B502AC44F8043D024612
:1006D4000B460348214602F0D6FC02B010BD00BF11
:1006E400110600004FF02002EFF3118382F311880A
:1006F400BFF36F8F0121044AC2F8401583F31188B8
:10070400BFF36F8F0020704700900350524A136864
:1007140043F0020313600022D30003F57F03D3F8F0
:100724000013013108D0D3F800130132D3F8043395
:10073400B2F5807F0B60EFD1484AD36913F001030F
:100744003BD0474B1946D3F80024012AFBD1C3F808
:100754000425D1F80034012BFBD1404BDA69D207D0
:1007640008D5DA693E4922F00102DA61D1F80024A1
:10077400012AFBD11A6A01320AD11A6A22F0FF0255
:1007840042F020021A62364AD2F80034012BFBD11F
:100794000022334BC3F80425D3F80024012AFBD1EB
:1007A400BFF34F8F2F49304BCA6802F4E062134302
:1007B400CB60BFF34F8F00BFFDE7126A0132C0D098
:1007C4002A4A116809290AD12949096801390129E4
:1007D4009EBF4FF05021C1F81431C1F8183113688D
:1007E400092B09D1224B1B68012B01BF214A13603D
:1007F400A2F63822C2F878351C4B1A68092A0BD1A4
:100804001B4A1268022A07D100211A4A11600121E9
:10081400A2F63822C2F878151B68092B06D1144BAE
:100824001B68022B02BF0C22134B1A600D4BD3F82A
:100834008C2042F44062C3F88C20D3F8882042F420
:100844007002C3F88820BFF34F8FBFF36F8F0B4B39
:100854000B4A1A60704700BFD0ED00E00080FF0033
:100864000090035000ED00E00400FA053001FF00A1
:100874003401FF00384A0050E4AE035074260020CF
:100884000090D00308B504464FF02002EFF3118323
:1008940082F31188BFF36F8F02F0A5FD204600F0AC
:1008A4004FFF034802F04BFD00F0ECFBFCE700BFF8
:1008B4000F3D00000A2838B50446074D04D12868C6
:1008C4000D2143685B6898472868E1B243685B6818
:1008D4009847204638BD00BF0800002010B5044CDE
:1008E400204601F0CFF82046BDE81040FFF7E4BEF3
:1008F400B908000008B5044801F0D8F9034B1860A2
:10090400FFF7ECFF002008BD383D00000800002080
:1009140010B54FF02003EFF3118283F31188BFF376
:100924006F8F154C237833B982F31188BFF36F8F1F
:100934006FF0440010BD013BDBB2237033B182F38E
:100944001188BFF36F8F6FF00F00F3E70B4B01219A
:10095400187838B1217082F31188BFF36F8F6FF06C
:100964000A00E7E7197082F31188BFF36F8F044A16
:1009740011601870DEE700BF1E1900201D19002049
:100984000450005010B54FF02002EFF3118382F3AE
:100994001188BFF36F8F144C207898B183F31188BA
:1009A400BFF36F8F4FF05022D2F81C34D2F81824C2
:1009B40003F0030343F48033934314BF6FF0430005
:1009C400002010BD0122227083F31188BFF36F8FC2
:1009D4004FF05023C3F80401C3F818150221C3F8DB
:1009E40004139A60DEE700BF1C190020F8B54FF02D
:1009F4002002EFF3118382F31188BFF36F8F294A2A
:100A04001078441C147080B183F31188BFF36F8F86
:100A14004FF05023D3F80C3403F00113B3F1011F4A
:100A24000CBF00206FF0430009E01F4D2F783FB149
:100A3400107083F31188BFF36F8F6FF00A00F8BD55
:100A440001262E7083F31188BFF36F8F4FF050246B
:100A540021B3052000F054FDC4F80071D4F8043328
:100A6400C4F804632660D4F800219AB10022DB079D
:100A740058BF0123C4F800214FF0200258BFC4F826
:100A840008330A4B0520C3F8802100F029FD002318
:100A94002B70BDE720BF40BF20BFE4E7C4F80011BE
:100AA4002660F4E71E1900201D19002000E100E073
:100AB4000022104B10B4C3F840214FF02002EFF392
:100AC400118482F31188BFF36F8F0B4AD3F80405A6
:100AD4001168401A20F07F4323F0FF030B44136096
:100AE40084F31188BFF36F8FC0F30F205DF8044BBC
:100AF40001F0D4BC005001500C00002038B51A4855
:100B040001F0D4F860B3436802211B6898470024BD
:100B14004FF48073154D4FF40012C5F80845C5F81D
:100B240040354FF48033C5F80433114B01211C6068
:100B3400104B1520C3F88021224600F0F5FC152047
:100B440000F0CEFC012320460B4A13602B60D5F83D
:100B5400043503F5807323F07F43C5F8403538BD71
:100B64004FF0FF30FBE700BF3F3D00000050015055
:100B74004051015000E100E00850015070B54FF6BB
:100B8400FE76B0F1FF3F08BF30464FF02003EFF38D
:100B9400118483F31188BFF36F8F421EB242A8BF42
:100BA4003246104D104BD5F804151B6822EAE27248
:100BB400C81A20F07F40FF3000EB022020F0FF0035
:100BC4000344591A21F07F411F2998BF03F580730C
:100BD40023F07F43C5F8403584F31188BFF36F8F4A
:100BE40070BD00BF005001500C0000204FF02002E7
:100BF400EFF3118382F31188BFF36F8F064AD2F8A3
:100C04000405064A1268801AC0F30F2083F3118882
:100C1400BFF36F8F704700BF005001500C000020DD
:100C240008B543B2002B0CDB012200F01F018A40FF
:100C34005B091049203341F82320BFF34F8FBFF3E2
:100C44006F8F830003F1A04303F540533128D3F899
:100C5400002806D0002A07DA02F00302023A012A29
:100C640002D8054AC3F80028002102F0F9FB00204D
:100C740008BD00BF00E100E00001008030B54FF482
:100C840080244FF0041585B04FF480212C4802F0E5
:100C940056FB21682B4802F052FB29682A4802F0CF
:100CA4004EFB10220021684602F089FC2368684646
:100CB40000930294FFF734FC0120FFF761FC00204D
:100CC400FFF74AFC0120FFF76FFC01210020FFF72A
:100CD40089FCFFF77DFC2C681C4802F030FB0820DF
:100CE400FFF79EFF24F00104BFF34F8FBFF36F8F14
:100CF4006408640020462146224623469FED140AD8
:100D0400DFED130A9FED121ADFED111A9FED102A81
:100D1400DFED0F2A9FED0E3ADFED0D3A9FED0C4A01
:100D2400DFED0B4A9FED0A5ADFED095A9FED086A81
:100D3400DFED076A9FED067ADFED057AFFF7C2FB68
:100D4400703E0000873E00009C3E0000BA3E00005A
:100D5400000000002DE9F843694802F0F0FA002190
:100D6400DFF8E481674F684D58F82140CA0301F564
:100D7400C07347F82340654802F500434E1C02F057
:100D8400DEFA634B14F0100F6249634808BF19463A
:100D940002F0D5FA14F0040F14BF72212D21284655
:100DA40002F0CDFA14F0020F14BF77212D2128464A
:100DB40002F0C5FA14F0010F14BF78212D21284642
:100DC40002F0BDFA14F4807F14BF6C212D21284653
:100DD40002F0B5FA514802F0B2FA202E3146C3D1DE
:100DE4004F4B484CC3F3C432C3F30E03C3F5004363
:100DF400C3F34313C4F80025C4F80435D4F800152C
:100E0400D4F804254748520102F099FA434802F005
:100E140096FA424802F093FA434802F090FA00210D
:100E2400DFF82881384E58F821504A0301F5E07361
:100E340044F823503D4802F500534F1C02F07FFA5A
:100E4400334B15F0100F3349334808BF194602F0ED
:100E540076FA15F0040F14BF72212D21304602F0EA
:100E64006EFA15F0020F14BF77212D21304602F0DF
:100E740066FA15F0010F14BF78212D21304602F0D7
:100E84005EFA15F4807F14BF6C212D21304602F0E8
:100E940056FA224802F053FA202F3946C3D10024CF
:100EA4001E4802F04CFA224802F049FA154B214D33
:100EB400DFF89C80DFF89C90C3F8C04405EBC406BF
:100EC400777955F83420002F14BF43464B4621460A
:100ED400194802F034FA57B91848013402F02FFACD
:100EE400172CEBD10D48BDE8F84302F028BA30794D
:100EF400FFF796FE08B11248EFE71248EDE700BF8E
:100F04007D3D000000300050B53D0000A03D0000D4
:100F1400663D00005D3D0000593E00007D4200003A
:100F2400E07F0000B83D0000FE3D0000203E0000D0
:100F3400343E0000A03B0000503E00005C3E000038
:100F4400633E00006B3E0000203B0000203B00009D
:100F5400723D00006A3D0000902908B5134639D15E
:100F64000A4601461D4801F003FBBDE808407146EE
:100F740072467346B7EE000AF7EE000AB7EE001A9F
:100F8400F7EE001AB7EE002AF7EE002AB7EE003AA1
:100F9400F7EE003AB7EE004AF7EE004AB7EE005A11
:100FA400F7EE005AB7EE006AF7EE006AB7EE007A81
:100FB400F7EE007A8EF3008C10B4F1EE10CA4FF6FF
:100FC4006074C0F6FF740CEA040CE1EE10CA10BCA5
:100FD400F44674476FF01500C7E700BF1000002007
:100FE40004488168406A884203D003494FF0805224
:100FF4000A607047DC18002004ED00E013498A6899
:101004004FF028001044EFF3098C80E8F01F2020F3
:1010140080F31188BFF36F8F0D4F4FF000664A6A5B
:101024008A603E60506E0023536680F3118804B5D5
:101034000648806802F048FABDE8044002F128003E
:1010440090E8F01F8CF3098870470000DC1800203A
:1010540004ED00E01EF0040F0CBFEFF30880EFF383
:101064000980816931F8021C11F0FF010229FFD0C7
:1010740001B502F01EFA01BD014910220A60704751
:1010840010ED00E0404080F3118830BF704700BF8E
:10109400404080F311884FF004007146014202D0B1
:1010A400EFF3098001D1EFF30880714601B500F038
:1010B40075F901BD01B572B60B4A106A00281EBF4E
:1010C4000021116202F0DEFA62B6EFF30580A0F1AE
:1010D40010004FEAC0000549014409C99847BDE81A
:1010E4000140034800470000DC1800207838000065
:1010F400E50F0000002320210348C2180133412BCF
:1011040082F80013F9D1704700E100E0094A0A4966
:10111400936809685866996608494B6843F0805398
:101124004B60002383F31188BFF36F8F9368986E2D
:10113400704700BFDC180020883C000000ED00E090
:1011440038B51B4C05461B4802F0F9F8A36AD906CA
:1011540002D5194802F0F3F8A36A1A0702D5174812
:1011640002F0EDF8A36A9B070ED5154802F0E7F8E4
:10117400616BA36A180607D5124802F0E0F81DB1A6
:10118400A36A23F08003A362094CA36ADA0702D599
:101194000D4802F0D4F8A36A9B0602D50B4802F06E
:1011A400CEF8A36AA36A002043F0FF03A36238BD0C
:1011B40000ED00E04D400000644000009840000055
:1011C400AC400000C5400000DC400000FC400000D2
:1011D40038B51E4C05461E4802F0B1F8A36AD9047E
:1011E40002D51C4802F0ABF8A36A1A0502D51A48C6
:1011F40002F0A5F8A36A9B050ED5184802F09FF8E3
:10120400A16BA36A180407D5154802F098F81DB11C
:10121400A36A23F40043A3620C4CA36A590502D5C4
:10122400104802F08CF8A36ADA0509D50E4802F0DA
:1012340086F8064A0020936A43F47F43936238BDDC
:10124400A36A9B04F5D50948F1E700BF00ED00E06F
:10125400BF3F0000D63F000098400000E83F000078
:10126400024000001840000034400000FC40000030
:1012740010B51C4C1C4802F062F8A36A9A0102D50E
:101284001A4802F05CF8A36ADB0102D5184802F0A0
:1012940056F8A36ADC0202D5164802F050F8114C45
:1012A400A36A180302D5144802F049F8A36A590343
:1012B40002D5124802F043F8A36A9A0302D51048F3
:1012C40002F03DF8074CA36ADB0302D50D4802F097
:1012D40036F8A36A00206FEA03436FEA1343A3625C
:1012E40010BD00BF00ED00E00C42000025420000EC
:1012F40039420000544200007F4200009E42000038
:10130400C4420000DF42000010B51A4C1A4802F033
:1013140016F8A1696369580602D5184802F00FF857
:101324006369D90707D5164802F009F8636943F0E1
:10133400FF03636110BD63699A0701D51148F3E7A0
:1013440063695B0701D51048EEE76369180701D5A7
:101354000E48E9E76369D90601D50D48E4E76369F6
:101364009A0601D50B48DFE763691B06DED50A48F8
:10137400DAE700BFD0ED00E02C4100004641000058
:10138400574100006E4100008D410000A94100005A
:10139400C7410000DD410000F84100003D4B70B53D
:1013A4005E6801F07F43B3F17F4F05460C465DD183
:1013B40011F0010041D048061BD42968364B374848
:1013C4000B44012B98BF296C01F0B9FF14F00804F9
:1013D400304B09D0EFF389855C6814F4006408D1BC
:1013E4002F4801F0ACFF41E0EFF388855B681905F5
:1013F400F6D4C6F30806F21E092A3FD8DFE802F045
:1014040005383A2D343E3E3E3E3C264801F097FFD7
:10141400204BDA6A920701D52348E2E7D86A10F034
:1014240080400AD0214801F08AFF214B1B784BB140
:101434000120FFF785FE06282BD02946BDE8704021
:1014440000F0B4B81B4B1B781BB10120FFF7C0FEA2
:10145400F1E7194B188884B214B1FFF709FFEAE7E2
:10146400164B58690028E8D0FFF74EFF0020E4E748
:101474000020DEE70020E9E71148B2E711481249ED
:10148400A6F110020F2ED8BF0146104801F057FFF5
:10149400ECE770BD00ED00E0A6ED05013943000066
:1014A400594300007E43000096430000B843000007
:1014B40028ED00E029ED00E02AED00E0D0ED00E0A9
:1014C400D84300000B430000204300000F440000F9
:1014D400024A536943F010035361704700ED00E082
:1014E40043B2002B08DB012200F01F0002FA00F0D7
:1014F400024A5B0942F82300704700BF00E100E0A4
:1015040043B2002B0DDB012200F01F0002FA00F0B1
:101514005B09044A203342F82300BFF34F8FBFF323
:101524006F8F704700E100E043B2002B01F101012D
:10153400A8BF03F160434FEA4111B8BF054BC9B2DC
:10154400ABBF03F5614300F00F0083F80013195497
:10155400704700BF14ED00E02DE9F0418C18884677
:1015640017461E4604220A9B0999054602F034F9DF
:1015740000220D49A4F1200323F0070321F0010107
:10158400C5E91322C5E91687996106991E60596059
:10159400079999600899D9604FF08071D961AB645B
:1015A4006A66BDE8F08100BF5730000038B50446D4
:1015B4000D4605281AD8DFE800F00319191315178A
:1015C4000D4801F0BCFE00F025FEAA6901460B4857
:1015D40001F0B5FE29462046BDE8384000F018B8B1
:1015E4000748EEE70748ECE70748EAE701460748FB
:1015F40001F0A5FEE7E700BF23440000C14400005A
:101604004344000069440000834400009E440000F9
:10161400052810B50CD000F003FE60B100F000FE08
:101624000C490D4B002808BF19460C4801F087FEF1
:10163400FFF728FDFCE700F003FE0028EED1084C7C
:101644000848A16801F07BFEA068BDE8104000F0E6
:101654000BB800BFFD440000014500001245000026
:10166400DC1800203245000038B505464FF0200351
:10167400EFF3118483F31188BFF36F8F02F08DF8B9
:101684000A4B9B68AB420BD1094B5A68C2F3080260
:1016940012B92046FFF73AFD5A6842F080525A6068
:1016A4002046BDE8384002F01FB800BFDC18002017
:1016B40000ED00E001F051FE202080F3118808487D
:1016C4004FF40061401880F30988EFF3148002217D
:1016D400084380F31488BFF36F8F00F007F800000D
:1016E400701E002030BFFFF7FDBF00BF114A08B5D0
:1016F400114B22F07F029A60BFF34F8FBFF36F8FBD
:10170400D3F8882042F4A002C3F888200B4A536817
:1017140023F040435360BFF34F8FBFF36F8F002319
:10172400E1EE103A00F002FB00F00AFBFFF7E2FCE6
:1017340000F038FB0000000000ED00E030EF00E0B6
:10174400BFF34F8F0549064BCA6802F4E0621343A6
:10175400CB60BFF34F8F00BFFDE700BF00ED00E09B
:101764000400FA0510B50E4B88B002930D4B0E4CD5
:1017740003930E4B08A8049302AB40F81C3D0C4A9B
:101784002346012100F002F900230793094B0121AC
:10179400E41A05A80593069400F002F908B010BDF8
:1017A40000000020000000000000012006000100ED
:1017B400000000200000002010B50B680C7A23F014
:1017C4001F0304F01F021A43CB68640923F01F03AC
:1017D400044943F0010343EA44038860CA600B618F
:1017E40010BD00BF90ED00E02DE9F04F8046894622
:1017F40014460027484D85B04F4507DA58F827307E
:101804005E68C6B31F2E05D86FF01504204605B0D8
:10181400BDE8F08FF206F7D1D3F800A01AF01F0F3D
:10182400F2D1504601F09DFB834606EB0A000138D5
:1018340001F097FB8345E7D11BF1160FE4D0631E3B
:101844005B45E1DBC5F808B0E86858F82710C5F82F
:1018540008B02E6920F01F00D1E900321A449842E2
:1018640046F01F0602F1FF3A18D1564505D15FFA3A
:101874008BF001F031FE0137BEE7C5F808B0EB6824
:1018840022F01F0203F01F031A43EA60E0B201F0E2
:1018940023FE10F1160FB7D0441CECE7C5F808B0CE
:1018A4002A69013B23F01F0302F01F02134356452C
:1018B400E0B22B61EBD001F00FFE10F1160FA3D0B4
:1018C400C5F808B0EA689DF80830013E62F30403E5
:1018D4008DF808302B699DF808205B0863F34712E4
:1018E4008DF8082058F827200130D2E9003213443B
:1018F400009323F01F031E44A6EB0A06C4B226F08D
:101904001F060F2C03963FF67FAF20466946FFF76C
:1019140053FF0134AFE700BF90ED00E00522034B15
:101924005A60BFF34F8FBFF36F8F704790ED00E0A5
:10193400BFF35F8F0022014B5A60704790ED00E0C7
:1019440070B50E4D2E68102E15D80024FFF7F0FF49
:101954000B4B0C4A1A63A64205D10B4B1E70FFF7C2
:10196400DDFF002070BD6968204601EB0411FFF71C
:1019740023FF0134EFE74FF0FF30F3E7E03A0000D4
:1019840090ED00E0AAFF44001F19002010B5034C9D
:101994002278FFF729FF207010BD00BF1F19002017
:1019A4002DE9F74F894607460026DFF89080DFF8D7
:1019B40090A0214C4E4519DAD7F804B0BBF1000FC2
:1019C40036D03B681846019301F0CBFA019B0546DB
:1019D4000BEB0300013801F0C4FA1423854203FB26
:1019E40006F306D06FF0150248F8032003B0BDE8F3
:1019F400F08F15F1160F48F80350F7D09AF800202D
:101A0400AA42F3DDA5604344A560E068197B60F356
:101A1400040119732169187B490861F3471018738D
:101A2400E26822F01F025A60226922F01F021A6142
:101A340001360C37BEE700BF90ED00E0F017002040
:101A44001F19002070B50C4B0E461C780546234622
:101A540000210A4A0F2B0BDD094B191D1868FFF7EB
:101A6400ABFE224631462846BDE87040FFF7BCBEB7
:101A7400936011610133EDE71F19002090ED00E040
:101A8400F0170020014B1860704700BF7826002033
:101A940070B54B79012B23D18B79032B20D1CC79D1
:101AA4002CB1012C1CD103689B681B79C3B10A7942
:101AB40012B1022A14D10E2247F6122603689B683B
:101AC4001D680B68B3426BD027D8B3F5965F61D01D
:101AD40012D8B3F5167F4DD005D8B3F5967F74D0E0
:101AE4006FF0220052E0B3F5966F50D0B3F5166F45
:101AF400F6D14FF41D233FE0B3F5615F4CD004D819
:101B0400B3F5165FECD1324B36E0B3F5964F45D0C2
:101B1400B3F5E14FE4D12F4B2EE0B3F5E13F48D0CC
:101B240012D84DF6C026B3423DD005D8B3F5164FB2
:101B3400D6D14FF41D031FE0B3F5614F36D0B3F592
:101B4400963FCDD1244B17E0B3F5E12F37D008D819
:101B5400B3F5613F30D0214EB342C1D14FF0806321
:101B64000AE0B3F5612F2DD01D4EB342B8D14FF02A
:101B7400805301E04FF41C33C5F8243583682243B5
:101B840003C9C5F86C2583E80300002070BD4FF439
:101B94009E23F1E7134BEFE7134BEDE7134BEBE712
:101BA4004FF40003E8E74FF46503E5E74FF46B03F4
:101BB400E2E74FF0EB73DFE74FF06C73DCE74FF0D5
:101BC400E863D9E74FF07063D6E74FF4A033D3E767
:101BD4000050270000C0750000903A0190D0030027
:101BE40040420F0000B0130000F03A0000A04E0085
:101BF400026870B59268174B14684FF400728568D8
:101C040003219A6009260022C3F82412C3F818227B
:101C1400C4F80C650626C4F8146580269E60C3F8D3
:101C24001C12C3F864220723C4F808351923294673
:101C3400C4F81035FFF72CFF58B90823C4F8003551
:101C44001D440123C4F81001C4F83455C4F83835D0
:101C5400236070BD00258450014B1B68184700BFEA
:101C640088260020014B1B68184700BF8C260020E3
:101C7400024B0A461B680021184700BF902600202B
:101C840070B50026084B53F82040013053F820501B
:101C9400A54200D870BD236820465B68984700B110
:101CA40066600C34F4E700BF743C0000104B70B560
:101CB40005461E460F4C9C4204D10E4CB44209D139
:101CC400002412E062681AB122681268AA420CD099
:101CD4000C34F0E763680BB90C34EFE7236828464B
:101CE400196801F01BFC0028F6D1204670BD00BF26
:101CF400FC2600209C26002008B50B4D4FF0200246
:101D0400EFF3118382F31188BFF36F8F01F082FD2B
:101D1400012104460228D8BF084601F08BFD2C623D
:101D2400FFF7B0F9EAE700BFDC1800200248034AD5
:101D34000021121A01F043BC000000202C190020DD
:101D440008B50648064A0749121A01F00BFCBDE81B
:101D54000840054A0549064801F004BC70260020E5
:101D6400102700209045000000000000904500006E
:101D74000000002008B50220FFF782FF074801F0A9
:101D8400DEFA0320FFF77CFF00F0A0FA01F0E2F88E
:101D9400034A137B23F00103137308BD5745000066
:101DA4007018002080B5444BA2B083F30888002546
:101DB400E023424C012784F82230E57725766576C6
:101DC400A576E576636A3E4E43F4E0236362636A74
:101DD40043F400236362A563E3689BB243F0BF63EB
:101DE40043F40833E360FFF773FBFFF745F94FF063
:101DF400FF33A362E36207AB29466C22184601F065
:101E0400DEFBB06028468DF82970FFF739FF3846AD
:101E1400FFF736FF2B4C00F0F1F92B4B74624FF4B3
:101E24008062CDE90473CDE90255CDE90055274B15
:101E34002749204600F030FA637B354623F004023C
:101E440013F01B0F627304D1A36913B9204600F089
:101E540003F9204B0026059301220F231E4FCDE9E1
:101E64000332CDE9016600961C4B4FF4A0721C4965
:101E7400384600F011FA7B7BEF6023F004037B7398
:101E8400184BC5E90633E1EE106AFFF76BFC0D4809
:101E9400AC6001F019FB0D4B134A184682F3098814
:101EA40063B64FF0000181F31188BFF36F8F0021F7
:101EB4000022002301F0CDF87026002000ED00E0A0
:101EC400DC1800207018002084450000791D0000F3
:101ED400301900208945000004180020FD1C000072
:101EE400301D0020F4180020301D0020EFF3058081
:101EF4000D2809D828B1054B586880F40060C0F358
:101F0400C02080F0010070470120FAE700ED00E0F6
:101F140008B5FEF76BFE054B054A1B680021184403
:101F240010611846BDE8084001F084BC1419002073
:101F3400DC180020F8B50D464FF02003EFF31184B0
:101F440083F31188BFF36F8F4FF400410027002201
:101F54000B4E0C4BC1FB00671A6130464FF47A32CA
:101F640000233946FEF7ECF8074B1860074B1D6059
:101F7400FFF7CEFF84F31188BFF36F8FF8BD00BF66
:101F8400FFE70300DC1800201419002010190020BA
:101F94004FF02003EFF3118183F31188BFF36F8FA8
:101FA400044B9A68D37B013BD37381F31188BFF34D
:101FB4006F8F7047DC180020094B03F1280282421E
:101FC40005D19B688B4202D14B7BDB0607D1D1E95B
:101FD40000231A600A6853600023C1E90033704784
:101FE400DC18002038B50D4C024604F1280001F03D
:101FF40094FB054600B9E568A3684AB95A7BD20642
:1020040006D1AA6922B9DA897F2A01D9636238BD67
:102014009D4201D0FFF77CFF6562F8E7DC180020E1
:1020240010B54FF02003EFF3118483F31188BFF34D
:102034006F8F084B01209A68D37B0133D373FFF76A
:10204400D1FF84F31188BFF36F8FBDE8104001F016
:102054005ABB00BFDC180020F8B54FF02003EFF3A3
:10206400118483F31188BFF36F8F164A114651F818
:10207400283F8B420CD05BB1D66A90F90E5093F98D
:102084000E70AF420BDCB34202D01B68002BF6D1BA
:10209400D36A01604360D36A1860D06205E05A686D
:1020A400C0E900325A6810605860437B43F0400333
:1020B40043730020FFF796FF84F31188BFF36F8FFB
:1020C400F8BD00BFDC180020F8B504464FF020032B
:1020D400EFF3118683F31188BFF36F8F194F014615
:1020E40007F128052846FFF767FFBB6A3A46AB426B
:1020F4000CD05BB1F86A94F90E1093F90E708F420C
:102104000BDC834202D01B68002BF6D1D36A256016
:102114006360D36A1C60D46205E05968C4E9003185
:1021240059680C605C60637B906843F040036373A0
:10213400031B58425841FFF755FF86F31188BFF33C
:102144006F8FF8BDDC1800201449154A10B58B6850
:102154001468A34203D1BDE81040FFF7D9BE0024A0
:102164001460104A1268BAB1DA897F2A14D80E4A68
:1021740093F90E40126894420EDB0C4A12689342A3
:102184000AD09A6942B90A69824203DC1846FFF709
:102194009BFFE0E7121A0A6110BD00BFDC180020A3
:1021A4000C19002014190020101900208C3C000088
:1021B40038B504464FF02003EFF3118583F31188FB
:1021C400BFF36F8F437B5A0607D501460948FFF7D3
:1021D400F3FE637B23F040036373074B9868031B90
:1021E40058425841FFF7FEFE85F31188BFF36F8F05
:1021F40038BD00BF04190020DC1800200021044B66
:10220400084603F12802C3E90A22FFF793BE00BF80
:10221400DC180020014B9868704700BFDC180020D0
:10222400EFF305800D2807D838B1044B586880F4C3
:102234000060C0F3C02070470120704700ED00E04B
:10224400024B9B68187B00F001007047DC180020EB
:1022540010B502464FF02003EFF3118483F3118885
:10226400BFF36F8F437B590704D484F31188BFF302
:102274006F8F10BD23F00403437301F085FA10B18E
:102284001046FFF7E9FE2146BDE81040014801F081
:102294001DBA00BF2019002030B587B00E9D04463A
:1022A40004950D9D03950C9D02950B9D01950A9D2A
:1022B4000095FFF751F9044B9B6813B9236607B0E7
:1022C40030BD1B6EFAE700BFDC1800202DE9F04F8B
:1022D400284E294DB04687B0B54205F130040FD3DE
:1022E400FFF756FE4FF400490027234C234EDFF836
:1022F40090A0444521D307B0BDE8F04FFFF790BE4E
:1023040054F8043C059354F8103C049354F8143CDA
:10231400039354F8183C029354F81C3C019354F86A
:10232400203C009354E90A2354E90C01FFF7B4FF5D
:1023340054F8303CDD642546CEE7616A4B1C04D07A
:10234400256821B92846FFF783FF3034D1E7B34627
:10235400BC46C9FB01BC4FF47A320023584661469F
:10236400FDF7EEFE5146421C05F1180000F052F84C
:10237400EBE700BFFC260020FC260020FFE703005B
:102384002B370000034B1B680BB9FEF72FBC002052
:10239400704700BF18190020036840B1084A52680A
:1023A400904204D01BB19A6881680A449A604268DA
:1023B400136003685A600023C0E90033704700BF0C
:1023C4009426002038B5104B1B78002B0F4B18BFF8
:1023D4004FF0FF301C6808BF6FF000409C420AD0E9
:1023E4004CB1A568FFF7CEFF281A00280ADBA468C1
:1023F400FFF7C8FF201A064B1B6913B19842A8BF08
:10240400184638BD0020F6E7201900209426002045
:10241400DC18002070B504461646C1604FF0200356
:10242400EFF3118583F31188BFF36F8FFFF7AAFFD2
:10243400012EACBF80190130174BA0601A689A4274
:1024440001D05E6832B95A68236062605A681460C9
:102454005C600BE09068A168884216DD411A9160C7
:102464005168C4E9002151680C6054601A689A42AA
:1024740006D0944204D1FFF7A5FF0021FEF77EFBAE
:1024840085F31188BFF36F8F70BD091A9642A1605E
:10249400D9D01268D6E700BF942600202DE9F04B6E
:1024A4000446FFF751FE4FF02003EFF3118583F349
:1024B4001188BFF36F8F214F214EB846DFF8849007
:1024C4003460D9F8004032684C45D7E900BC05D0E7
:1024D40024B1A368934214DD9B1AA36000241BEB70
:1024E40002004CEBE271C8E900013460FFF76AFFB7
:1024F4002146FEF743FB85F31188BFF36F8FBDE8D8
:10250400F08B1BEB03004CEBE371D31A3360002315
:10251400C7E90001A3602046FFF73EFF85F3118859
:10252400BFF36F8FE36898474FF02003EFF31185F3
:1025340083F31188BFF36F8FC3E700BF000000204F
:10254400181900209426002038B5074C074DAC42DA
:1025540001D3002038BD04F114032046C4E9053337
:1025640000F02CFD1C34F2E7FC260020FC260020A1
:102574002DE9F04192B00592002966D0002B64D079
:10258400002A62D00F461D460446E0B106AE30462E
:10259400042100F0BFF808A8282100F0BBF808A81F
:1025A40000F066F8002841D020464FF4BF51FFF7F1
:1025B4005FFB4FF0FF3530460421FFF759FB2846F7
:1025C40012B0BDE8F0814FF4BF510120FFF744FB86
:1025D4008046002839D006AE3046042100F09AF82F
:1025E40008A8282100F096F808A800F041F802464F
:1025F400002834D107ABCDE902800093019508A9E6
:1026040005AB304600F0A8FB48BB2A68059B9A42FC
:102614001ED94FF0FF354FF4BF514046FFF728FB5A
:10262400002CC8D14046FFF71DFBC4E707ABCDE93A
:10263400024002460093019508A905AB304600F01C
:102644008BFBA0460028AFD1DFE74FF0FF35B6E79C
:1026540007993846083100F05BF80025DBE74FF4B2
:10266400BF514046FFF704FB4FF0FF35DAE700BFE8
:102674001C2330B583B002A941F8043D044600F0A0
:102684004DF80546D8B9019B1C2B1BD1D4E9003267
:1026940001210033E16118BF01230AB143F00203B1
:1026A400A26832B9E268AAB9C4E908323BB90D4D4F
:1026B40009E0E26843F0040362B9C4E90832284639
:1026C40003B030BD084D20461C2100F023F82846F5
:1026D40003B030BD0022284643F00803C4E90832A1
:1026E40003B030BD0E0CF000370CF000BFF34F8F79
:1026F4000549064BCA6802F4E0621343CB60BFF39A
:102704004F8F00BFFDE700BF00ED00E00400FA05B5
:1027140000F011BF0A46002100F051BF18B111B1F9
:102724000B681C2B01D0012070474FF47F033A4AF9
:10273400D3F8101C91425AD0D3F8102C013256D041
:10274400D3F8102C4FF47F030260D3F8141C334ADF
:1027540091425ED0D3F8142C01325AD0D3F8142C01
:102764004FF47F034260D3F8182C12F5947F4DD0B8
:10277400D3F8182C013249D0D3F8182C4FF47F0326
:102784008260D3F81C1C264A91423CD0D3F81C2CFE
:10279400013238D0D3F81C2C4FF47F03C260D3F835
:1027A400002C70322DD0D3F8002C013229D0D3F86C
:1027B400002C4FF47F030261D3F8042CAF321ED0F7
:1027C400D3F8042C01321AD0D3F8042C4FF47F032D
:1027D4004261D3F8081C134A91420BD0D3F8082C59
:1027E400013207D0D3F8083C83610020704740F6DB
:1027F400FC02A7E740F2373383610020704751227F
:10280400E4E79022D5E742F60412C5E740F6D86221
:10281400B4E742F2D002A3E7FCF8FFFFD020FFFFA9
:102824000429FFFF37F3FFFFA8B32DE9F0414C1E45
:10283400B4F5047F2CD25BB352B34FF0000CC90043
:10284400E646654664464F1E03F1FF380CE0AB4292
:1028540016D08E4501D10CF1010CA84516D00134D7
:10286400BC4205F1010518D8610950F8211004F0A3
:102874001F06F1401F2E18BF01F00101002CE6D104
:102884000025A8458E464FF0010CE8D16245E6D2FA
:102894000348BDE8F081024870470020BDE8F0819C
:1028A400370CF1002DE9F04F8FB00D46DDE91941E9
:1028B4008346002959D129690391002104F5C16097
:1028C4001860189B1960002A00F02281814A824B0B
:1028D40011686A6A1B689A4257D10A2955D19BF834
:1028E400033006930399042308467C4A0293A2FB0F
:1028F40000029208CB0002EB420204F5C260A1EB95
:102904004202013BDFF8D091DFF800A2049000926C
:102914000593189B039C1C60002C00F0CC800026BF
:10292400049F00F0F1FA00230793069BBBF1000F0C
:102934003AD0002D34D053BB5B000693BBF1000F9B
:1029440036D0002D34D0E3B106A9284600F0CCFAE5
:10295400002800F07D81624B984212D0009000F074
:10296400D3FA00980FB0BDE8F08F4FF47F01D1F88F
:102974000C0C01300CBF4FF40471D1F80C1C039102
:102984009BE72B6A73B95648E8E75648E6E706A979
:10299400284600F0A9FA68B1534B9842DED0069B52
:1029A400082BC9D15148D9E7082BFBD05B0006930B
:1029B4004F48D3E72946069800F078FA0028EBD16F
:1029C400069B082B00F00E81042B00F03181A3F14B
:1029D4000203B3FA83F35B09019301231946454AC1
:1029E400136042F8843C434B19606B6AC9F80030A9
:1029F400D9F800206B6A9A42F5D14FF000084FF0E5
:102A0400FF30CAF8008000F027FA3B4A3B4B4046AF
:102A14001A6000F02FFA0A22019839492D4B0860F8
:102A24001A602A69A8F15538A8FB02126B6A1209C8
:102A340003EB4303DB0303FB02F3324A9B091360FA
:102A44000123CAF800300699DBF800200B0243EAA0
:102A5400016322F07F421343CBF8003007A800F053
:102A640015FA002898D1284BA8FB04281A681433B7
:102A7400089253F8102CB6EB980F099253F80C2CCB
:102A84000A9253F8082C0B9253F8042C0C921B68EE
:102A94000D9301D1009B9BB93846182208A9FFF772
:102AA40037FE183C18370136002C7FF43AAF049BEC
:102AB400002B40F09A800023189A1360069B6FE75E
:102AC4001A46384608A9E41AFFF722FE009B1F4461
:102AD400E9E700BF3811845030118450ABAAAAAA88
:102AE400310CF100300CF100020CF100320CF10059
:102AF400350CF100C4118450FEFFFF0F0011845007
:102B04000C118450D8118450141184502C11845009
:102B1400BBF1000F3FF44CAF002D3FF449AF01234C
:102B24000EA941F8203DCBF80020284600F0DCF93E
:102B340000287FF413AF2946069800F0B7F900285F
:102B44007FF40CAF069F082F00F0EB80042F00F0F9
:102B5400EA80A7F10207B7FA87F77F090122164630
:102B6400734B74491A6018460A60943B06606A6A9B
:102B74001A6019686A6A9142F8D14FF000086E4BE6
:102B84004FF0FF30C3F8008000F066F96B4B6C4ADD
:102B940040461A6000F06EF90A226A496A4B0F60D7
:102BA4001A601A992B6901296A6A00F0B180674991
:102BB400A1FB03131B09012102EB4202D20303FB15
:102BC40002F3634A9B0913605B4B19600699DBF8B7
:102BD40000200B0243EA016322F07F421343CBF847
:102BE40000307FE603230193F7E6039BB3F5047FEC
:102BF4003FF661AFDDE9047C204623466E6904E0BC
:102C0400012001336345144615D85A0957F8222088
:102C140003F01F01CA401F2918BF02F00102002B54
:102C2400EED0A242ECD101308642EAD149480BE011
:102C340002230193D1E64FF48063DDE90310AA690E
:102C4400FFF7F2FD00285DD00023189A1360A3E675
:102C54002946069800F02AF900287FF47CAE069CE9
:102C6400082C51D0042C51D0A4F10204B4FA84F4F9
:102C7400640901231E4619462D4A136042F8843C18
:102C84002B4B19606B6AC9F80030D9F800206B6AC5
:102C94009A42F5D100274FF0FF30CAF8007000F0D7
:102CA400DBF8264B264A38461A6000F0E3F80A227D
:102CB4002449254B0C601A602A6924496B6AA1FBDC
:102CC400021203EB43031209DB0303FB02F3204A62
:102CD4009B091360CAF80060069BDBF800101A0217
:102CE40042EA036321F07F421A43130A03F47F0389
:102CF400134323F07F43CBF80030029B013B029344
:102D04007FF407AE002029E60324B2E70224B0E7EB
:102D14004FF47F03D3F80C1C013106D0D3F80C3CDC
:102D240045E703271AE7022718E7162343E700BFFE
:102D3400C4118450401184502C11845000118450CB
:102D4400FEFFFF0F0C11845038118450ABAAAAAABD
:102D5400D8118450360CF1002DE9F0431B4C85B09A
:102D64000746DDE90D56884620684FF0FF3191464D
:102D740000F036F828BB002000F036F8E8B900234C
:102D8400CDE9005602934A46414638460C9BFFF76C
:102D940089FD0546012000F027F850B9206800F0AD
:102DA40021F810B10A48FFF7A1FC284605B0BDE898
:102DB400F0830848FFF79AFCF0E70748FFF796FC12
:102DC400DDE70648FFF792FCD5E700BF2419002091
:102DD400E83C0000C83C0000A83C0000903C000017
:102DE4000020704700207047194B82B0D3E8AF2F02
:102DF4000192019A98B90132D3E8EF1FC3E8E02F9A
:102E04000028F9D18A42F7D1BFF35F8F019B1BB928
:102E14000122104BC3F80025002002B07047002A9D
:102E2400FAD0019A012A0ED0019A013AD3E8EF1F91
:102E3400C3E8E02F0028F9D18A42F7D1BFF35F8FAE
:102E4400002002B070470021024AC2F80015EBE7E7
:102E54002819002000008450430503D54FF0FF32A9
:102E6400024B1A60024B1860704700BF081184506F
:102E7400081A8450014B1860704700BF041A84502C
:102E840008B100F04FB84FF47500704708B501461B
:102E94004FF48060FFF7F4FF00230249024A0B60FD
:102EA400136008BDC81184502C11845001380728C0
:102EB40015D8DFE800F0100C140814141404CB68BF
:102EC40000204B6270478B6800204B6270474B6850
:102ED40000204B6270470B6800204B62704701482A
:102EE400704700BF310CF1000B6802E0082B0B6047
:102EF40006D8026A13424FEA4303F7D00020704712
:102F040000487047310CF10000230449044A0B6067
:102F14004FF480601360FFF79FBF00BF2C118450F3
:102F2400C41184500246074803681342FCD021B1FF
:102F3400054B06481B680B600360054B00201A60B4
:102F4400704700BF001A8450041184500811845043
:102F5400081A845008B5FDF7FDFEBDE80840FDF7EA
:102F64008DBE40E800F313F4803FD8B208BF6FF081
:102F74001500704770B50C254D43C66890F90B00D9
:102F840074198842A8BF21464FF0200492FBF4F440
:102F9400B8BF715902F01F0001EB8401196070BDC4
:102FA40007B501ABFFF7E6FF0123019A03FA00F02E
:102FB40013680343136003B05DF804FB2DE9F84381
:102FC4000446FF2200214FF00C0E43680589006877
:102FD4005D4394F80AC02844E2728C4505DC002560
:102FE4002389AB4222DCBDE8F883B5FBF3F20EFB88
:102FF40001F7D4F80C801F2A08EB0706C8BF1F325C
:103004004FEA930306F10409C8BF520903F103030D
:10301400C6E9019923F00303D4BFE17248F807001D
:1030240001F10101C8BF00EB8200D6E76268E368E2
:103034006A4320681E1D811886509A6820464A609B
:103044009A68116099602A460021FFF7A9FF0135AB
:10305400C6E708B50446084611461A46A047FFF7D6
:10306400D9F8FEF701FB0020704770B50D46044601
:103074004520A04729465220A04729462346BDE8BB
:103084007040522018472DE9F04F4FF0000A0646D1
:103094000F464FF0FF39D04689B01C46531E0393A8
:1030A400002505E06DB9252800F03D813946B0477B
:1030B400039B13F8010F03930028F3D109B0BDE873
:1030C400F08F642862D019D839280AD8312851D20F
:1030D4002D283DD030283ED0252808D13946B04788
:1030E400DEE7582800F0A880632800F016813946EE
:1030F4002520B047039B39461878F0E7702800F084
:10310400918006D8692841D06C283CD06828CFD05B
:10311400EDE775286DD017D87328E8D1256804F138
:10312400040B2B461C4614F8010B002840F0EC80DD
:10313400B8F1030F40F000815C1BA9EB0404002CE0
:1031440000F3E6805C46ABE7782875D07A28DEE7A2
:103154004FF00308ACE7B9F1000F0EDAB8F1000F35
:1031640000F0E780A0F13009B8F1000F08BF4FF07C
:1031740002089DE7B9F1000FF4DB0A2303FB0909F8
:10318400A9F13009F0E70AF1010A91E7BAF1000F59
:1031940012D125680434002D05DA39462D20B047B4
:1031A4006D4209F1FF3943462A46CDF8009039466D
:1031B4003046FDF733FA73E7BAF1010FE9D04FF067
:1031C400000C4FF0FF3B073424F0070303F108041D
:1031D400D3E9002312F1004043F100018C4508BFFC
:1031E400834504D239463046FFF73FFF58E715467A
:1031F400D1E7BAF1000F05D122680434CDF800906C
:103204004346D4E7BAF1010FF6D0073424F007039C
:1032140003F10804D3E90023002B08BFB2F1004FE7
:10322400ECD3DFE739463020B04739467820B04741
:103234004FF008094FF00108BAF1010F27DC2368A9
:10324400043407930023049310220023934602932B
:103254000693079B0BF1FF3B4FEA8B00C0F1200C58
:10326400A0F1200123FA00F0049B03FA0CFC40EACD
:103274000C0023FA01F1084310F00F0013D1069B50
:1032840013B9BBF1000F2ED14FF0300C11E007340D
:1032940024F007031A6803F108045B680792049397
:1032A400D2E7059AD5E709288CBF4FF0570C4FF0A9
:1032B400300C394660440592B047029B06950133B1
:1032C4000293BBF1000FECD1B8F1030F7FF4E8AE29
:1032D400029BC3EB4905002D7FF7E2AE394620205F
:1032E400B047013DF7E7531E91450593E9DBB8F17B
:1032F400010F03D139463020B047E2E7B8F1020F9D
:10330400DFD139462020F7E73946B047234609E79D
:1033140039462020B047013C11E72068251D394675
:10332400B0472C46BCE6AA46A8464FF0FF39012513
:10333400BEE64FF00108BBE65C460546B8E60FB4AE
:1033440007B504A951F8040B0191FDF7BBF903B0CB
:103354005DF804EB04B070477047FDF7D7B94FF040
:10336400502330B5D3F80851D3F80423D3F80041DF
:1033740002F00102D3F80413D3F8040115B10025B7
:10338400C3F80851B4B14FF050230024C3F80041EE
:1033940022B14FF050230122C3F8082348B1002280
:1033A4004FF05023C3F804218A0702D50222C3F840
:1033B400082330BD002AF1D04FF05023D3F80C3449
:1033C40003F00113B3F1011FE8D1E2E708B50022CD
:1033D40001210520FEF7A8F80520FEF781F800205A
:1033E40008BD70477047704708B50120FDF74AFAD9
:1033F400BDE808407046714672467346B7EE000A4F
:10340400F7EE000AB7EE001AF7EE001AB7EE002A3C
:10341400F7EE002AB7EE003AF7EE003AB7EE004AAC
:10342400F7EE004AB7EE005AF7EE005AB7EE006A1C
:10343400F7EE006AB7EE007AF7EE007A8EF3008CAE
:1034440010B4F1EE10CA4FF66074C0F6FF740CEAC3
:10345400040CE1EE10CA10BCF4467447FDF718BE24
:1034640043B2A9B1002B12DB01215B099B0003F1DC
:10347400604303F56143D3F8802200F01F0001FA92
:1034840000F022EA0000C3F88002D3F880327047CB
:10349400002BFCDB01225B099B0003F1604303F575
:1034A4006143D3F8801200F01F0002FA00F00843D1
:1034B400E9E701460068FEF779B808B5FEF712F9A6
:1034C400BDE80840FDF78CBD07B5002101A8FEF753
:1034D400B9FA03B05DF804FB30B54B6885B00C68ED
:1034E4009DF808200D890094498924F01F04013BAC
:1034F400234465F3040261F3471223F01F030F28EA
:103504008DF808200393044605D86946FEF754F95C
:10351400204605B030BD6FF01504F9E701380139D4
:1035240010F8013F11F8012F934202D1002BF7D17B
:103534001A46981A7047431A934210B500EB0203D7
:1035440008D3024601399A420BD011F8014F02F810
:10355400014BF8E70A4412F8014D8A4203F8014D81
:10356400F9D110BDF0B581EA0004A50703460BD0DC
:10357400013B0A4491421DD1F0BD002AFCD011F850
:10358400014B013A03F8014B9C07F6D10C461D1F71
:103594008F183E1B032E08D86FF00305940805FB13
:1035A4000422A40023442144E2E754F8046B45F8C0
:1035B400046FEEE711F8014B03F8014FDAE7034615
:1035C400F0B5C9B29C070FD11D4641EA012444EA73
:1035D40004449F187E1B032E0CD8940803EB840428
:1035E40013449C4209D1F0BD002AFCD003F8011B0E
:1035F400013AE7E745F8044BECE704F8011BF0E770
:103604004FF0FF3070470B46826892E8030083E86E
:1036140003000020704703689B681B68D3F82401EB
:1036240018B1D3F88004C3F8800470470368826833
:103634009B681B68D3F8100138B1127A00200A7015
:103644000122C3F810011A6070474FF0FF30704731
:1036540082B002AA02F8011D002103689B681B685E
:10366400C3F82011C3F844250122C3F848259A6001
:10367400D3F820110029FBD0DA6002B07047002093
:1036840070477047FFF7AEBE437BDB0603BF80691C
:10369400B0FA80F040090020704738B504464FF076
:1036A4002003EFF3118583F31188BFF36F8F014675
:1036B4008068FEF781FC637B23F00203637385F368
:1036C4001188BFF36F8F0023A36038BD08B5FEF7E0
:1036D4000DFC20B1BDE808400846FDF717BD81F395
:1036E4001188BFF36F8F08BD08B50246FEF7FEFBD5
:1036F40020B1BDE808401046FDF708BD82F31188EB
:10370400BFF36F8F08BD4FF02003EFF3118083F3F5
:103714001188BFF36F8FFFF7E7BF0368984214BFA8
:1037240018460020704750F8103C70B50446A0F1CC
:103734001805CBB14FF02003EFF3118683F3118802
:10374400BFF36F8F294650F8100CFEF735FC14F8C0
:103754000B3C23F0020304F80B3C86F31188BFF3FF
:103764006F8F002344F8103C14F80B3C284623F0D8
:10377400140304F80B3CFFF787FF20B12846BDE88B
:103784007040FEF769BC70BD437BDB0603BF8069F4
:10379400B0FA80F0400900207047036D10B504466C
:1037A40003B198472046FFF7EFFF38B12046FEF7F4
:1037B400FFFC637B43F00803637310BD637B9B07CB
:1037C40002D52046FFF769FFA369002BF1D004F16D
:1037D400180000F009F8ECE70373002342738173C7
:1037E400C373C0E90633704710B54FF02002EFF3FE
:1037F400118482F31188BFF36F8F03683BB1FEF726
:10380400CBFD002084F31188BFF36F8F10BD6FF0E0
:103814001500F7E710B54FF02003EFF3118483F39D
:103824001188BFF36F8FFEF7CDFD84F31188BFF3CA
:103834006F8F10BD70B504460E464FF02003EFF3B2
:10384400118583F31188BFF36F8FFEF7BBFDA04290
:1038540005DD012803DD31462046FDF78FF985F3A8
:0A3864001188BFF36F8F70BD70472D
:02386E00FFFF5A
:0838700074C9FF7F0100000094
:103878000000000061340000000000006134000016
:103888000000000061340000000000006134000006
:1038980000000000613400000000000063330000F5
:1038A80000000000613400000000000061340000E6
:1038B80000000000613400000000000061340000D6
:1038C80000000000613400000000000061340000C6
:1038D80000000000613400000000000061340000B6
:1038E80000000000613400000000000061340000A6
:1038F8000000000061340000000000006134000096
:103908000000000061340000000000006134000085
:10391800000000006134000000000000B50A00004B
:103928000000000061340000000000006134000065
:103938000000000061340000000000006134000055
:103948000000000061340000000000006134000045
:103958000000000061340000000000006134000035
:103968000000000061340000000000006134000025
:103978000000000061340000000000006134000015
:103988000000000061340000000000006134000005
:1039980000000000613400000000000061340000F5
:1039A80000000000613400000000000061340000E5
:1039B80000000000613400000000000061340000D5
:1039C80000000000613400000000000061340000C5
:1039D80000000000613400000000000061340000B5
:1039E80000000000613400000000000061340000A5
:1039F8000000000061340000000000006134000095
:103A08000000000061340000000000006134000084
:103A18000000000061340000000000006134000074
:103A28000000000061340000000000006134000064
:103A38000000000061340000000000006134000054
:103A48000000000061340000000000006134000044
:103A58000000000061340000000000006134000034
:103A68000000000061340000000000006134000024
:083A78000000000061340000B1
:103A8000653D0000E906000000000000653D000003
:103A9000F9080000000000003F3D0000D1330000A5
:103AA00000000000493D0000D1330000000000008C
:103AB000533D0000010B000000000000653D0000C8
:103AC0004519000000000000383D0000F51B000013
:103AD0006C3C0000653D00004D250000000000002A
:103AE00002000000E83A000000000000003D000075
:103AF00006000000E0FF0F0000000020083D00006D
:103B000021000000E0FF0020890900000000000003
:103B100000000000F109000015090000000000008D
:103B20001701000017010000170100001701000035
:103B30001701000017010000170100001701000025
:103B40000701000007010000070100000701000055
:103B50000701000007010000070100000701000045
:103B60000701000007010000070100000701000035
:103B70000701000007010000070100000701000025
:103B80000701000007010000070100000701000015
:103B90000701000007010000070100000701000005
:103BA000E53E000042010000EC3E0000050100007F
:103BB000F63E000015010000FF3E00003901000044
:103BC000083F000009010000133F00000A00000048
:103BD0001E3F00000A010000283F00000B0100000A
:103BE000323F00000F0100003D3F000010010000C7
:103BF000483F000011010000533F00000E0100008B
:103C00005D3F000021010000663F0000220100002E
:103C10006F3F000023010000783F000024010000F6
:103C2000813F00002A010000893F00003A010000A6
:103C3000913F00002C010000993F00001C01000092
:103C4000A23F00001D010000AB3F00003101000059
:103C5000B73F000018010000313600005536000063
:103C60001B360000951A00000B3600000080005043
:103C7000010000009C260020F0260020FC260020E9
:103C8000FC260020FC260020F5FFFFFF0418002082
:103C90004661696C20746F2061637175697265207B
:103CA0006D757465780A00004661696C20746F2038
:103CB000696E63726561736520504D20636F756E28
:103CC0007465720A000000004661696C20746F2000
:103CD000646563726561736520504D20636F756E16
:103CE0007465720A000000004661696C20746F20E0
:103CF00072656C65617365206D757465780A000086
:103D0000464C4153485F30005352414D5F300046AE
:103D100061696C656420746F207265626F6F743ABC
:103D2000207370696E6E696E6720656E646C657372
:103D3000736C792E2E2E0A00554152545F30004389
:103D40004C4F434B5F33324B00434C4F434B5F313F
:103D5000364D007379735F636C6F636B00536563FB
:103D60007572650909004E6F6E2D53656375726536
:103D700009004E6F6E2D53656375726500466C6168
:103D8000736820726567696F6E0909446F6D6169B8
:103D90006E09095065726D697373696F6E730A00FD
:103DA0002530327520307825303578203078253030
:103DB00035782009002563004E6F6E2D736563759D
:103DC00072652063616C6C61626C65207265676905
:103DD0006F6E203020706C6163656420696E2066B0
:103DE0006C61736820726567696F6E202564207747
:103DF0006974682073697A652025642E0A0053521D
:103E0000414D20726567696F6E0909446F6D616984
:103E10006E09095065726D697373696F6E730A007C
:103E200025303275203078253035782030782530AF
:103E3000357809005065726970686572616C0909AE
:103E4000446F6D61696E09095374617475730A007A
:103E500025303275202573090925730009534B4914
:103E6000500A00094552524F520A00094F4B0A00AE
:103E700053504D3A204E5320696D6167652061743F
:103E800020307825780A0053504D3A204E53204D6B
:103E9000535020617420307825780A0053504D3AF1
:103EA000204E5320726573657420766563746F725B
:103EB00020617420307825780A0053504D3A2070E4
:103EC00072657061726520746F206A756D70207400
:103ED0006F204E6F6E2D53656375726520696D613D
:103EE00067652E0A004E52465F5030004E52465FC4
:103EF000434C4F434B004E52465F52544331004EA9
:103F000052465F4E564D43004E52465F5541525405
:103F10004531004E52465F554152544532004E5293
:103F2000465F5457494D32004E52465F5350494DFB
:103F300033004E52465F54494D455230004E524672
:103F40005F54494D455231004E52465F54494D45EC
:103F50005232004E52465F5341414443004E524656
:103F60005F50574D30004E52465F50574D31004E16
:103F700052465F50574D32004E52465F50574D33B8
:103F8000004E52465F495043004E52465F564D43E5
:103F9000004E52465F465055004E52465F454755CB
:103FA00031004E52465F45475532004E52465F47FC
:103FB00050494F544531004E52465F574454002AF1
:103FC0002A2A2A2A20425553204641554C54202A59
:103FD0002A2A2A2A0A002020537461636B696E67BB
:103FE000206572726F720A002020507265636973D7
:103FF00065206461746120627573206572726F72EE
:104000000A00202042464152204164647265737365
:104010003A20307825780A002020496D7072656357
:1040200069736520646174612062757320657272C2
:104030006F720A002020496E737472756374696F21
:104040006E20627573206572726F720A002A2A2AC6
:104050002A2A204D5055204641554C54202A2A2AC0
:104060002A2A0A002020537461636B696E672065F9
:1040700072726F722028636F6E746578742061723B
:104080006561206D69676874206265206E6F7420B9
:1040900076616C6964290A002020556E737461632F
:1040A0006B696E67206572726F720A00202044612E
:1040B0007461204163636573732056696F6C61742A
:1040C000696F6E0A0020204D4D46415220416464C4
:1040D000726573733A20307825780A002020496E83
:1040E000737472756374696F6E2041636365737373
:1040F0002056696F6C6174696F6E0A002020466CEF
:104100006F6174696E672D706F696E74206C617A6F
:10411000792073746174652070726573657276615D
:1041200074696F6E206572726F720A002A2A2A2AD9
:104130002A20534543555245204641554C54202A88
:104140002A2A2A2A0A002020416464726573733A7D
:1041500020307825780A002020496E76616C6964E9
:1041600020656E74727920706F696E740A00202069
:10417000496E76616C696420696E746567726974F2
:1041800079207369676E61747572650A0020204931
:104190006E76616C696420657863657074696F6EB2
:1041A0002072657475726E0A002020417474726901
:1041B000627574696F6E20756E69742076696F6CB4
:1041C0006174696F6E0A002020496E76616C6964C3
:1041D000207472616E736974696F6E0A0020204CDE
:1041E000617A792073746174652070726573657289
:1041F000766174696F6E0A0020204C617A792073B1
:1042000074617465206572726F720A002A2A2A2A04
:104210002A205553414745204641554C54202A2ACF
:104220002A2A2A0A0020204469766973696F6E2061
:104230006279207A65726F0A002020556E616C6980
:10424000676E6564206D656D6F727920616363656B
:1042500073730A002020537461636B206F7665725C
:10426000666C6F772028636F6E7465787420617256
:104270006561206E6F742076616C6964290A002084
:10428000204E6F20636F70726F636573736F72205F
:10429000696E737472756374696F6E730A0020209F
:1042A000496C6C6567616C206C6F6164206F66207F
:1042B0004558435F52455455524E20696E746F20E5
:1042C00050430A002020496C6C6567616C2075734F
:1042D00065206F662074686520455053520A00209F
:1042E00020417474656D707420746F206578656307
:1042F00075746520756E646566696E656420696EA7
:10430000737472756374696F6E0A005265736572B7
:1043100076656420457863657074696F6E20280047
:1043200053707572696F757320696E7465727275FA
:1043300070742028495251200020205320696E7348
:104340007472756374696F6E2061646472657373EF
:104350003A2020307825780A00524554544F424183
:10436000534520646F6573206E6F74206D617463B4
:1043700068204558435F52455455524E0A002A2A38
:104380002A2A2A2048415244204641554C54202A8A
:104390002A2A2A2A0A002020427573206661756C39
:1043A00074206F6E20766563746F72207461626C26
:1043B0006520726561640A0020204661756C742076
:1043C000657363616C6174696F6E20287365652025
:1043D00062656C6F77290A002A2A2A2A2A204465F6
:1043E000627567206D6F6E69746F722065786365A2
:1043F0007074696F6E20286E6F7420696D706C65C3
:104400006D656E74656429202A2A2A2A2A0A002AE0
:104410002A2A2A2A20257320256429202A2A2A2AA2
:104420002A0A002A2A2A2A2A20486172647761729D
:104430006520657863657074696F6E202A2A2A2A60
:104440002A0A002A2A2A2A204B65726E656C2041AE
:104450006C6C6F636174696F6E204661696C757214
:104460006521202A2A2A2A0A002A2A2A2A2A204BB7
:1044700065726E656C204F4F505321202A2A2A2ADC
:104480002A0A002A2A2A2A2A204B65726E656C2085
:1044900050616E696321202A2A2A2A2A0A002A2AC0
:1044A0002A2A20556E6B6E6F776E20466174616CA0
:1044B000204572726F7220256421202A2A2A2A0A36
:1044C0000043757272656E74207468726561642051
:1044D0004944203D2025700A4661756C74696E67F9
:1044E00020696E737472756374696F6E20616464A1
:1044F00072657373203D20307825780A0049535245
:1045000000657373656E7469616C207468726561AF
:104510006400466174616C206661756C7420696E1C
:1045200020257321205370696E6E696E672E2E2EC2
:104530000A00466174616C206661756C7420696E56
:1045400020746872656164202570212041626F7259
:1045500074696E672E0A002A2A2A2A2A20426F6F5F
:1045600074696E67205A6570687972204F5320769F
:10457000312E31342E39392D6E637332202A2A2A96
:104580002A2A0A006D61696E0069646C650000008A
:104590006B3000000090D0030536000000C201001F
:1045A0000001030000000000833600008736000091
:0C45B000C3350000942600209426002053
:1045BC00803A00000000000000000000D43A000027
:1045CC000000000000000000BC3A000000000000E9
:1045DC0000000000983A0000083B000000000000BA
:1045EC00A43A0000143B000000000000C83A000090
:1045FC00583C00007C2600208C3A00000000000093
:10460C0000000000B03A00000000000000000000B4
:10461C00FC260020FC26002000000000000000000A
:04462C000F0000007B
:10463000FFFFFFFFFFFFFFFFFFFFFFFFFFFFFFFF8A
:10464000000000000000000000000000000000006A
:10465000000000000000000000000000000000005A
:10466000000000000000000000000000000000004A
:107FE0007FE97FE9F8F7BABF7FE97FE9FBF7FEB9E0
:107FF0000000000000000000000000000000000081
:04000003000016B92A
:00000001FF
